:100000000C94A3060C94CB060C94CB060C94CB0654
:100010000C94CB060C94CB060C94CB060C94CB061C
:100020000C94CB060C94CB060C94CB060C94C11DFF
:100030000C94CB060C94CB060C94CB060C94CB06FC
:100040000C94E22D0C94CB060C94CB060C94CB06AE
:100050000C94CB060C94CB060C94CB060C94CB06DC
:100060000C9489190C94CB06070792282810381293
:1000700092070782287C2854288207078224580088
:10008000344882070782483400502C820707825484
:1000900054545454820707822828282828820707A6
:1000A00082101010101082070700447C28447C0046
:1000B000070700547C28283800401E00000000007C
:1000C0000000000000000000000000000000000030
:1000D00000000000006C00000000003FFF93FFF8EC
:1000E000007C003FFF93FFF801FF0000006C000060
:1000F00003838000000000000701C0000000000032
:100100000C0060000000000018003000000000003B
:1001100018003004081020403000180E1C3870E021
:100120003000181B366CD9B03FFFF831E3C78F1889
:100130003FFFF820C1830608000000000000000017
:100140000000000200008000100000070001C00055
:10015000380000070001C0003800000F8003E000F5
:100160007C0000070001C000380000071FF1C3FE3B
:1001700038FF80070FE1C1FC387F000F87C3E0F82C
:100180007C3E000F87C3E0F87C3E000F87C3E0F899
:100190007C3E000F8FE3E1FC7C7F001FDFF7F3FE66
:1001A000FEFF800000000000000000496E76616CD8
:1001B0006964206D6F7665210043616E2774206D40
:1001C0006F76652070696563652E004D6F76696E88
:1001D00067206261636B776172647321004E6F20E8
:1001E0006D6F766520666F7220796F752E004E6F89
:1001F000206D6F76652E2043505520736B697073A8
:100200002E00436F6E6E656374696F6E206C6F7342
:1002100074000A0A5072657373201520746F20638E
:100220006F6E74696E75652E000A4E657874207461
:1002300075726E20666F723A0A00436F6D6D2E20E4
:100240006572726F720031206D6173746572206D1A
:100250006178210057616974696E6720666F72204A
:10026000636F6E6E6563742E2E00436F6D6D756ED9
:1002700069636174696F6E204572726F720020202D
:100280002D3D2D20434F4E54524F4C53202D3D2D8C
:100290000A153A206D6F76652070696563650A18E6
:1002A000191A1B3A206D6F76652073656C6563744F
:1002B000696F6E0A20686F6C64201920746F206764
:1002C0006574206E65787420706F737369626C65F5
:1002D000206D6F76650A173A206261636B20746F38
:1002E000206D656E750A00A6034004E104720514D2
:1002F00006AE062507B0073408D9086309710979E5
:10030000097E09870953656E6574004350550043A3
:100310006C6F73653A150043505520574F4E005986
:100320004F5520574F4E0047414D45204F5645529F
:10033000210091099F09AC0954696D656F75743A84
:10034000204E6F20636F6E6E65637400B309BF0942
:10035000CB094F4B3A1500163A43616E63656C004A
:10036000596F7572205069656365733A005069650D
:100370006365732070657220506C617965723A0014
:1003800047616D65204D6F64653A00202D3D2D203D
:1003900047414D45205345545550202D3D2D2000BB
:1003A00053656E657400202D3D2D2053454E4554F8
:1003B00020494E54524F202D3D2D0A53656E6574D1
:1003C00020697320616E206F6C642067616D652009
:1003D000706C617965642062792065766572796FE9
:1003E0006E6520696E20616E6369656E7420456775
:1003F0007970742E205573696E672070726F706506
:100400007220626F6172647320616E64207069652E
:10041000636573206F72206A757374207468652039
:1004200073747265657420616E6420736F6D6520EE
:1004300073746F6E6520616E6420776F6F642E0039
:10044000202D3D2D2053454E45542052554C4553AB
:10045000202D3D2D0A53544152543A204561636882
:1004600020706C61796572206765747320332D3755
:100470002070696563657320706C616365642061D9
:100480006C7465726E6174696E67207374617274E6
:10049000696E672061742073717561726520312EF9
:1004A0000A4D4F56453A20342074776F2D73696496
:1004B000656420706164646C65732061726520748A
:1004C00068726F776E20746F2064657465726D69F1
:1004D0006E652074686520706C6179657227732081
:1004E000006D6F76657320666F72206F6E65207089
:1004F000696563652E0A4D6F76696E67206469725F
:10050000656374696F6E3A0A7C317C3E7C3E7C3E4A
:100510007C3E7C3E7C3E7C3E7C3E7C767C7C767C5D
:100520003C7C3C7C3C7C3C7C4F7C3C7C3C7C3C7CF8
:100530003C7C7C3E7C3E7C3E7C3E7C3E7C567C7E95
:100540007C3E7C3E7C497C7E3A20547261703B202C
:100550004F3A20486F757365206F66205265626957
:100560007274683B20493A207371333020476F61C1
:100570006C00207768697465202B202020202020C3
:100580002B7468726F770A207369646573202B6D12
:100590006F766573202B616761696E0A20202031B8
:1005A0002020207C2020203120207C205965730AC7
:1005B000202020322020207C2020203220207C205F
:1005C0004E6F0A202020332020207C202020332042
:1005D000207C204E6F0A202020342020207C2020E8
:1005E000203420207C205965730A202020302020D0
:1005F000207C2020203620207C205965730A283456
:100600007820626C61636B203D3E2036206D6F76F2
:1006100065732900596F75206D6F7665206167617C
:10062000696E206966207468726F77696E672061F1
:1006300020312C2034206F7220302E0A4154544136
:10064000434B3A204C616E64696E67206F6E206187
:100650006E206F70706F6E656E74732720706965A1
:10066000636520697320616E2061747461636B2C13
:10067000616E6420796F752065786368616E676567
:1006800020706C616365733B20796F75206D6179B3
:10069000206E6F74206C616E64206F6E20796F75B0
:1006A00072206F776E207069656365732E00524506
:1006B000535452494354494F4E533A0A2D46697296
:1006C0007374206D6F7665206D757374206D6F7611
:1006D0006520746865207069656365206F6E2068A9
:1006E000696768657374207371756172652E0A2D70
:1006F0005361666520737175617265733A20313597
:100700002C2032362C20323820616E642032392081
:1007100063616E6E6F742062652061747461636BD7
:1007200065642E0A002D446566656E63653A205443
:10073000776F206F72206D6F7265206F70706F6EB3
:10074000656E742070696563657320696E20612031
:10075000726F772063616E6E6F74206265206174C2
:100760007461636B65642E0A2D426C6F636B616408
:10077000653A205468726565206F72206D6F7265EE
:10078000206F70706F6E656E74207069656365733D
:1007900020696E206120726F772063616E6E6F74C6
:1007A000206265207061737365643B202D3E2000DC
:1007B00020686F776576657220626C6F636B616429
:1007C000657320646F206E6F7420207475726E20C4
:1007D00061726F756E6420636F726E6572732E0A3C
:1007E0002D547261703A204C616E64206F6E2073DC
:1007F0007175617265203230206D65616E73206D98
:100800006F76696E67206261636B20746F20746815
:100810006520666972737420656D707479207371D8
:1008200075617265206265666F72652073712E3125
:10083000362E0A002D457869743A20596F75206D5F
:100840006179206E6F74206D6F76652070617374AE
:100850002033302E2041207069656365206F6E2043
:1008600033302063616E2062652072656D6F76653E
:1008700064206174205354415254206F6620796F74
:100880007572207475726E20696620616C6C2079B7
:100890006F75722070696563657320617265206F82
:1008A0007574206F6620666972737420726F772E7C
:1008B0000A2D4E6F204D6F76653A20496620796F7C
:1008C000752063616E6E6F74206D6F766520666F44
:1008D0007265776172642C200020796F75206D75C8
:1008E0007374206D6F7665206261636B77617264EB
:1008F00020286163636F7264696E6720746F20746F
:1009000068652073616D652072756C6573292E2092
:100910004966206E6F206D6F766520697320706F59
:10092000737369626C652C20796F757220747572AF
:100930006E20656E64732E0A0A57494E3A20596F2D
:10094000752077696E2062792072656D6F76696EA9
:100950006720616C6C20796F7572207069656365C2
:10096000732E00506C6179202F20526573756D6570
:1009700000526573746172740048656C7000436F57
:100980006E74726F6C73004D61696E204D656E758B
:1009900000486F737420286D617374657229004A72
:1009A0006F696E2028736C617665290043616E6300
:1009B000656C00202073696E676C65202020002024
:1009C00020206D756C7469202020006D756C746931
:1009D0002028693263290003053F213F1208120ACB
:1009E000100A0E1C0E0C1E0C141A14161F161E13C1
:1009F0001E1E1B1E1E1F1E3F213F3A2F3A173D177A
:100A00003F213F181F02040A041F0E04040E1F0A90
:100A10001F0A0E0E1F04110E2E252E2F2A2E2629F8
:100A200029021F02081F08150E04040E150E1515C5
:100A30001B151B040604040C04000000001700032F
:100A400000031F0A1F16371A1904130A153A000368
:100A500000000E11110E000A040A040E04003000FA
:100A60000404040010001804031F111F121F101D9E
:100A7000151711151F07041F17151D1F151D01013F
:100A80001F1F151F17151F000A00003200040A114E
:100A90000A0A0A110A040115020E11171E051E1F6B
:100AA000150A0E110A1F110E1F15111F05010E1137
:100AB0001D1F041F111F1108100F1F041B1F1010F2
:100AC0001F061F1E040F0E110E1F09060E112E1FEA
:100AD000051A121509011F011F101F0F180F1F0CF7
:100AE0001F1B041B031C03191513001F11030418FB
:100AF000111F000201022020200001020C121E1F03
:100B0000120C0C12120C121F0C1A14041E05242AAB
:100B10001E1F021C141D1020201D1F0814111F1061
:100B20001E041E1E021C0C120C3E0A040C123E1E59
:100B3000040214160A020F120E101E0E100E1E08CA
:100B40001E120C1226281E322A26041E21001F0007
:100B5000211E040102013F213F45006801000005FC
:100B6000006801380100000500380168010000F646
:100B7000E8DBCFC3B8AEA49B928A827B746E6862B6
:100B80005C57524E4945413E3A3734312E2C292785
:100B90002523211F1D1C1A191716151413121110C5
:100BA0000F0E0D0C0B0A09080706AE0BB20B010164
:100BB000F7030101FF030A4E6F2053442063617263
:100BC00064206F720A6E6F204C4F414445522E488C
:100BD00045580A0A153A45786974001D20466C612B
:100BE0007368696E670A20206C6F616465722E2ECF
:100BF0002E0A0A444F4E2754205455524E204F4639
:100C00004621006D560A0A504C454153450A545539
:100C1000524E204F4646004C4F57204241545445B7
:100C200052590A00177361766500166261636B00A2
:100C30001574797065000A0A0A153A6F6B6179209C
:100C4000163A6564697400596F7520656E74657233
:100C500065640A00540A03E181867F3E186D830FA4
:100C60000F0E0183866033186DC3198F1803C38E6E
:100C70006033186DE330CF1803C39E603630CDE388
:100C800060CF3006C79E7E3E30CDB360CF300CC6FD
:100C9000F6603330D9B660CF33CFCCF66061B0DBCD
:100CA0001E60CF30D86CE6C061B0DB1E618F199832
:100CB0006CC6C063B19B0E330F0FB078C6FF7E1FAA
:100CC0001B061E0F1753440016137800161314004A
:100CD00015102000152010000000050089300802C2
:100CE0003802497868140000000000002400270042
:100CF0002A0000000000250028002B000000000052
:100D0000230026002900040404040404040402024D
:100D1000020202020303030303030102040810207A
:100D20004080010204081020010204081020000085
:100D3000000700020100000304060000000000009C
:100D40000000DF0B001811241FBECFEFD8E0DEBF7C
:100D5000CDBF11E0A0E0B1E0ECEAF8E602C00590FA
:100D60000D92AC32B107D9F714E0ACE2B1E001C0AA
:100D70001D92A33BB107E1F71DE0C6E4DDE004C02E
:100D80002297FE010E941934C234D107C9F70E948C
:100D90005A300C9454340C940000A0E0B0E0E3ED21
:100DA000F6E00C942534EC01A880B980CA80DB8081
:100DB000A114B104C104D10441F484E2A82E89ED48
:100DC000B82E8BE5C82E87E0D82EC601B5012DE1DF
:100DD00033EF41E050E00E94FC3327EA31E440E089
:100DE00050E00E9488337B018C01C601B5012DE1E2
:100DF00033EF41E050E00E94FC33CA01B9012CEE10
:100E000034EF4FEF5FEF0E9488336E0D7F1D801F20
:100E1000911F97FF04C061507040804090486883E4
:100E200079838A839B839B01AC015F77B901CA01F7
:100E3000CDB7DEB7EAE00C9441340E94CD060895A8
:100E400087E091E00E94CD060895609307017093BA
:100E500008018093090190930A010895982F8A3020
:100E600011F481E0089580E0943109F481E008955F
:100E7000262F30E023703070220F331F6695669561
:100E8000FC01E60FF11D83E090E0022E02C0880F06
:100E9000991F0A94E2F780956281862350E043709F
:100EA000507002C0440F551F2A95E2F7842B8283AD
:100EB0000895262F26952695FC01E20FF11D8281CB
:100EC00090E070E063707070660F771F02C09595B8
:100ED00087956A95E2F783700895813021F082301A
:100EE00021F481E0089582E0089580E00895DC0116
:100EF000FB012281E081121644F48E2F8F5F33278D
:100F000027FD30952E0F311D0EC04E2F50E041159C
:100F1000510511F480E002C08E2F8150332727FD48
:100F20003095240F351F2E31310514F02DE130E0BE
:100F3000722F582F60E02FC05A3011F0543109F44D
:100F400060E0852F86958695FD01E80FF11D2281D1
:100F50001A968C911A97813021F0823021F441E069
:100F600003C042E001C040E030E0852F90E0837094
:100F70009070880F991F02C0359527958A95E2F7E2
:100F80002370241711F060E005C06F5F633010F02C
:100F900081E008955F5F751778F680E00895CF933C
:100FA000DF93EC01A62FB0E0862F86958695FE0193
:100FB000E80FF11D228130E0CD0183709070880F21
:100FC000991F02C0359527958A95E2F7237009F499
:100FD0003EC0241709F43DC06E30D9F16931C9F122
:100FE0006B31B9F16C31C9F534C0862F81505D97F2
:100FF00014F06DE101C06F5F582F70E026C0852F9F
:1010000086958695FE01E80FF11D22818A85813043
:1010100021F0823021F441E003C042E001C040E011
:1010200030E0852F90E083709070880F991F02C088
:10103000359527958A95E2F72370241711F070E013
:1010400003C0713031F071E05F5F6517C0F681E079
:1010500001C080E0DF91CF910895109731F680E0D4
:10106000CACF0F931F93CF93DF93EC018B0188813D
:101070009981FB012081892B61F440E030E088896F
:1010800090E0880F991F01972817390771F541E003
:101090002CC0FB016281620F6E3128F54381862FDF
:1010A00086958695FE01E80FF11D228130E0862F9E
:1010B00090E083709070880F991F02C03595279536
:1010C0008A95E2F72370241771F0CE010E94CF07B2
:1010D000882349F0CE01B8010E94770790E0882369
:1010E00019F491E001C090E0492F842FDF91CF9156
:1010F0001F910F910895CF92DF92EF92FF920F937D
:101100001F937C016B01FB016181862F869586957B
:10111000F701E80FF11D028110E0862F90E0837047
:101120009070880F991F02C0159507958A95E2F770
:101130000370F6018081282F26952695F701E20F8E
:10114000F11D428150E090E083709070880F991FEC
:1011500002C0559547958A95E2F74370C7010E94F2
:101160003807C701F6016081402F0E943807F70158
:1011700017861F910F91FF90EF90DF90CF90089509
:10118000EF92FF921F93CF93DF93EC017B011EE060
:10119000812F86958695FE01E80FF11D228130E0B2
:1011A000812F90E083709070880F991F02C0359551
:1011B00027958A95E2F72370C9F4488550E0B4E09A
:1011C00055954795BA95E1F74370CE01612F0E947E
:1011D0003807CE016AE140E00E943807F701118329
:1011E000DF91CF911F91FF90EF9008951150D0CFD4
:1011F000EF92FF920F931F93CF93DF937C01EB014C
:101200000E943108882361F16A818881680F6983AF
:10121000862F86958695F701E80FF11D028110E073
:10122000862F90E083709070880F991F02C01595EB
:1012300007958A95E2F70370C7014B810E94380732
:10124000C7016881402F0E94380781E0F701878736
:1012500089818A3139F4C701BE010E94C00802C0E9
:10126000F7011786F7018785DF91CF911F910F91C5
:10127000FF90EF900895BC01655F7F4F0E94F808D2
:101280000895CF93DF93EC018F858823A9F5898595
:1012900090E09595879595958795682F63708A85D9
:1012A000681751F540E050E0842F86958695FE0141
:1012B000E80FF11D828190E09A0123703070220FB7
:1012C000331F02C0959587952A95E2F7837086179C
:1012D00099F04F5F5F4F4A30510531F7CE016DE114
:1012E00040E00E9438078A85FE01E80FF11D8189E0
:1012F0008F5F818B81E001C080E0DF91CF91089505
:10130000DC0120E0FC01E60FF11D918950968C91E3
:10131000981709F421E0822F0895EF92FF920F931E
:101320001F93CF93DF937C01EB010881102F21C025
:10133000812F86958695F701E80FF11D228130E017
:10134000812F90E083709070880F991F02C03595AF
:1013500027958A95E2F723708B81281749F4188323
:10136000C701BE010E943108882311F081E005C049
:101370001F5F1E31E8F2088380E0DF91CF911F915B
:101380000F91FF90EF900895FF920F931F93CF93CB
:10139000DF938C01EB01F88018820E948D0988236D
:1013A00091F48A8181958A83C801BE010E948D09CA
:1013B000882349F4F8828A8181958A8381E0F80143
:1013C000878780E001C081E0DF91CF911F910F916D
:1013D000FF900895FC0187858823B9F085858430C6
:1013E00079F0863069F0813059F08285813021F0C2
:1013F000823021F481E003C082E001C080E0828776
:10140000808191810196918380830895DF92EF928C
:10141000FF920F931F93CF93DF93EC01D62EE62E0E
:10142000FF24EE0CFF1C00E00DC0102F1F5FCE014B
:10143000602F41E00E9438070E5FCE01612F42E02D
:101440000E943807802F90E08E159F0574F31E2DA3
:1014500006C0CE01612F40E00E9438071F5F1E3199
:10146000C0F31982188281E08F8782E08A87D88A48
:101470001A8A1B8ADF91CF911F910F91FF90EF90F5
:10148000DF9008950F931F9310E000E00E94200763
:1014900060FD1F5F0F5F0430C9F7112309F416E0E8
:1014A000812F1F910F910895CF93DF93EC018F85CA
:1014B000882339F00E94420A8D871B868A858E8791
:1014C0001F86DF91CF9108956F927F928F929F92A6
:1014D000AF92BF92CF92DF92EF92FF920F931F9342
:1014E000CF93DF933C01862ECC24DD24EE24992477
:1014F00000E010E0AA24BB24F02EC301602F0E945C
:1015000059078E1509F058C0EE2009F455C0802FF8
:101510000E942E07882309F04FC09394C3016F2DBA
:101520000E945907E82E2CE12F1550F03BE1F316ED
:1015300068F48EE0F81651F099E1F91649F406C006
:101540002DE1F21629F4C2E2D1E003C0E50101C0A9
:10155000E80131E0391550F4892D90E09E01289F73
:10156000E001299FD00D389FD00D1124E81419F403
:10157000CC0EDD1E07C0882D0E946D07E81611F401
:10158000CC1ADD0A0F5F1F4F83E090E0A80EB91E52
:101590000E31110509F0B0CFC601DF91CF911F9137
:1015A0000F91FF90EF90DF90CF90BF90AF909F9002
:1015B0008F907F906F9008959924B0CFBF92CF9273
:1015C000DF92EF92FF920F931F93CF93DF93EC0183
:1015D0009BE0E92EF12CEC0EFD1ECE01B7010E941E
:1015E000C409882349F1C12C80E8D82ECE010E947D
:1015F0003B09CE016A850E94640A8C018A850E949B
:101600006D07682FCE010E94640A9801281B390BD0
:10161000C216D30614F4BB846901CE01B7010E943F
:101620007B088B858F5F8B87CE01B7010E948D0968
:101630008823E1F6BB8681E0DF91CF911F910F9166
:10164000FF90EF90DF90CF90BF900895FC01742F32
:10165000643508F05DC047FD5BC040330CF058C0F6
:10166000878D823019F5842F8595859585959927E5
:1016700087FD9095462F552747FD509524E530E08E
:10168000829FF001839FF00D929FF00D1124E40FD3
:10169000F51FEE54FD4F808190E0272F277002C088
:1016A000959587952A95E2F780958170972F959566
:1016B00095959595462F552747FD5095272F2770CF
:1016C0008823A1F4E4E59E02F0011124E40FF51F44
:1016D000EE54FD4F81E090E002C0880F991F2A95DB
:1016E000E2F780952081282320830895E4E59E0277
:1016F000F0011124E40FF51FEE54FD4F81E090E05E
:1017000002C0880F991F2A95E2F72081282B208399
:101710000895DB01FA016EE10E94A7339A3058F474
:101720008AE08083892F90E033E0880F991F3A95F3
:10173000E1F7029610C0292F30E0943170F482E175
:1017400080838AE090E0821B930B23E0880F991F2F
:101750002A95E1F7865B8C9308958AE1808383E084
:10176000220F331F8A95E1F72E5930402C930895AC
:10177000262F63E00E94A733392F822F6AE00E9450
:10178000A733292F313019F489E0891B282F8AE0EB
:10179000389FC0011124820F0895282FFB01DA0120
:1017A0006AE00E94A7338083822F0E94A7339C9314
:1017B0008081813019F489E0891B8C930895ECE2D3
:1017C000F1E086E8DF011D928A95E9F710927D012C
:1017D00010927C0187E291E090937B0180937A01E3
:1017E00008951F931092440111E08CE291E00E9451
:1017F00068208823D1F386E391E064E00E94C92C3D
:10180000882371F486E391E065E00E94C92C882367
:1018100039F486E391E066E00E94C92C882349F000
:1018200081E591E00E94E51D81E0809344011F91D4
:1018300008951092830110928401109381018AE728
:1018400091E06EE772E00E94E330CFCF0F931F93D9
:101850001092440110E001E08CE291E00E946820C7
:101860008823D1F386E391E065E00E94C92C8823A8
:1018700041F486E391E066E00E94C92C882309F4D4
:1018800041C081E591E00E94EB1D81E0809344011D
:101890001F910F91089581E591E00E94F11D1123A0
:1018A00011F419E01CC011501AC086E391E062E007
:1018B0000E94C92C882339F486E391E064E00E94F9
:1018C000C92C882361F081E591E00E94F11D812FF0
:1018D00090E001966AE070E00E94C733182F1092E2
:1018E00083011092840100938101E12FF0E0EE0F5B
:1018F000FF1FE951FD4F659174918AE791E00E94C5
:10190000E330AACF86E391E060E00E94C92C8823EF
:1019100009F0C1CFCACF0F931F9302E312E0C801B1
:1019200062E070E00E948B17C8016AE10E944818CB
:10193000C8010E948B181F910F91089582E392E0D5
:1019400062E070E00E948B1782E392E060E80E9400
:10195000481882E392E00E948B1882E392E062E0F2
:1019600070E041E050E00E949C18882329F082E357
:1019700092E00E949E1781E0089582E392E062E087
:1019800070E00E948B1782E392E068E10E944818A1
:1019900082E392E00E948B1882E392E062E070E0C2
:1019A00041E050E00E949C18882311F420E008C018
:1019B00082E392E00E949E1720E0892B09F021E04B
:1019C000822F089582E392E062E070E00E948B171C
:1019D00082E392E068E20E94481882E392E00E946B
:1019E0008B1882E392E062E070E041E050E00E94F8
:1019F0009C18882331F082E392E00E949E17809326
:101A0000CB0108950F931F9305E011E041C01092A0
:101A10008301009384018AE791E064E572E00E940B
:101A2000E33082E392E062E070E00E948B1782E391
:101A300092E060E80E94481882E392E00E948B18CE
:101A400082E392E062E070E041E050E00E949C1886
:101A50008823F1F082E392E00E949E178034910582
:101A600069F08038910569F41092B4018CE291E03C
:101A700066E472E044E10E943E1E1DC01093B40172
:101A800007C08CE291E06AE372E044E10E943E1EEE
:101A90008091B401882379F486E391E066E00E94A6
:101AA000C92C882341F48CE291E00E9468208823AD
:101AB00009F4B7CFACCF1F910F9108950F931F93E7
:101AC00002E312E0C80162E070E00E948B17C801D7
:101AD00064E20E9448186091CB01C8010E94481836
:101AE000C8010E948B181F910F91089582E392E024
:101AF00062E070E00E948B1782E392E061E10E9455
:101B0000481882E392E00E948B1882E392E062E040
:101B100070E044E150E00E949C18882341F082E389
:101B200092E067EB71E044E150E00E949530089547
:101B30000F931F9302E312E0C80162E070E00E947D
:101B40008B17C80160E10E944818C80167EB71E07B
:101B500044E150E00E941718C8010E948B181F91A1
:101B60000F91089582E392E062E070E00E948B178B
:101B700082E392E061E30E94481882E392E0609180
:101B8000C7010E94481882E392E00E948B1882E30A
:101B900092E062E070E00E948B1782E392E068E3DB
:101BA0000E9448186091CC0182E392E00E9448189C
:101BB00082E392E00E948B1882E392E062E070E0A0
:101BC0000E948B1782E392E062E30E94481882E34E
:101BD00092E061ED71E04AE050E00E94171882E364
:101BE00092E00E948B1882E392E062E070E00E9433
:101BF0008B1782E392E065E30E94481882E392E04B
:101C00000E948B1882E392E062E070E04AE050E0CC
:101C10000E949C18882349F082E392E06BED71E00A
:101C20004AE050E00E94953008951092B401089562
:101C30001092E6018091E5018832A9F0893228F4FA
:101C4000813151F08831A9F52DC0853389F0803874
:101C5000E9F0833371F511C082E392E067EB71E044
:101C600044E150E010C06091CB0182E392E01EC0DD
:101C700082E392E06BED71E004C082E392E061EDFB
:101C800071E04AE050E00E94171808958091B30176
:101C9000882321F082E392E060E808C082E392E0CA
:101CA00060E404C082E392E06091C6010E9448189B
:101CB00008958CE291E06AE672E044E10E943E1EE3
:101CC000089582E392E00E94A01808958091E601B1
:101CD0008F5F8093E6018091E601823058F0809119
:101CE000E601853038F461E070E080E090E00E9429
:101CF0005E2EECCF8091E60190E0823008F491E016
:101D0000892F08951092E60182E392E00E949E17C7
:101D10008093E5018091E501813309F1823348F434
:101D20008A3109F448C0843299F0803109F04CC0FE
:101D300008C0843351F1883389F1823309F044C0FB
:101D40001FC082E392E067EB71E044E150E023C002
:101D500082E392E00E949E178093CB01089582E374
:101D600092E00E949E17682F87EB91E00E94060A7E
:101D700081E080930B018093B6018093B4010895B4
:101D800082E392E061ED71E004C082E392E06BEDEA
:101D900071E04AE050E00E949530089582E392E0BD
:101DA0000E949E178093CC018091CC010E946D0708
:101DB0008093CD01089510920B0181E080930C0176
:101DC0001092CF011092D00108950F931F9302E358
:101DD00012E0C80162E070E00E94BF18C80162E82A
:101DE0007EE00E94F617C80168E17EE00E94FB17C2
:101DF0001092E5011F910F9108950F931F93DF93A8
:101E0000CF9300D0CDB7DEB78B01BE016F5F7F4FA0
:101E1000AE014E5F5F4F0E94890B8AE791E06981B6
:101E20004A8198010E94E2290F900F90CF91DF9193
:101E30001F910F910895DF92EF92FF920F931F93DE
:101E4000CF93DF9312E0A6EFEA2EAFEFFA2EC9EFA1
:101E5000DFEFF0E3DF2E8CE291E00E946820882320
:101E6000D1F386E391E064E00E94C92C882379F4E1
:101E700086E391E065E00E94C92C882341F486E363
:101E800091E066E00E94C92C882309F47BC081E5BB
:101E900091E00E94E51DDF91CF911F910F91FF907E
:101EA000EF90DF9008958AE791E06FE173E004C05E
:101EB0008AE791E067E173E00E94E33020917E01C0
:101EC00030E0C901880F991F820F931F909581956B
:101ED0009F4F8C5A9F4F62E070E00E94C73360931F
:101EE000830140917F0150E0440F551F440F551F5F
:101EF0004E5F5F4F40938401E091CC01F0E0E954E4
:101F0000FE4F2189205D8AE791E001E00E94632A6B
:101F10006091830180917E01680F609383018AE75D
:101F200091E0409184012AE30E94632A6091830139
:101F300080917E01680F60938301E091CD01F0E014
:101F4000E954FE4F2189205D8AE791E040918401A8
:101F50000E94632A81E08093820180917E018C9FA0
:101F6000802D11248C5A8093830180917F019D2DB7
:101F7000981B909384018AE791E06FE073E00E94E0
:101F8000E33069CF1093820180917E018E9D802D78
:101F90001124865D80938301109384018AE791E088
:101FA00067E273E00E94E33080917F0190E0019648
:101FB000880F991F8093840180917E018C9F802DD2
:101FC0001124865D809383016091CC0187EB91E0C1
:101FD0000E948009882309F066CF6ACF0F931F9370
:101FE0001092830181E08093840110E011C08AE7A0
:101FF00091E0609183014091840101E00E94632A95
:102000001F5F8091830190917E01890F80938301EE
:10201000E12FF0E0EF52FE4F2081222341F7909113
:10202000CC018091C101891799F4109283014091EC
:10203000840180917F01480F4093840120917E01AB
:10204000129F202D11248AE791E060E00E94B127C1
:102050008091B201882311F000E02DC020917E0113
:1020600030E0C901880F991F820F931F90958195C9
:102070009F4F8F5A8093830181E0809384018AE788
:1020800091E06BE073E00E94E3309091CD0180918C
:10209000C101891709F043C080917E0190E09C0145
:1020A000220F331F280F391F66277727621B730BF8
:1020B0006F5A28C00F5FE02FF0E0E552FE4F80819D
:1020C0008823C1F780917E01089F802D112411E59E
:1020D000912F981B9093830181E0809384018AE77C
:1020E00091E06BED71E00E94E2319091CD01809121
:1020F000C1018917A1F420917E01029F202D112496
:10210000612F621B609383014091840180917F0164
:10211000480F409384018AE791E00E94B127209103
:102120007E0130E0C901880F991F820F931F90959F
:1021300081959F4F8C5A9F4F62E070E00E94C73399
:102140006093830184E280938401E091CC01F0E00C
:10215000E954FE4F2189205D8AE791E044E201E0E5
:102160000E94632A6091830180917E01680F6093D1
:1021700083018AE791E0409184012AE30E94632A67
:102180006091830180917E01680F60938301E091EB
:10219000CD01F0E0E954FE4F2189205D8AE791E00E
:1021A000409184010E94632A1F910F910895CF925C
:1021B000DF92EF92FF921F93DF93CF9300D0CDB7C2
:1021C000DEB719E08AE791E061E0412F21E50E9446
:1021D000B127185F1932B1F711E08AE791E0612F5A
:1021E0004AE028E10E94BB27185F1935B1F710E0DB
:1021F00082E0C82ED12CCC0EDD1E7E010894E11C9D
:10220000F11C87EB91E0612F0E945907813009F49E
:1022100048C0813020F0823009F04CC046C01A31ED
:10222000B9F01B3130F41E3059F0193109F042C0B9
:102230000BC01C3161F11C3130F11D31D9F52DC0BD
:102240008EE068E670E026C089E161E770E022C0B8
:1022500060919C0170919D0180919E0190919F01E0
:1022600024E130E040E050E00E94DA336A3071054A
:102270008105910520F08AE16AE770E00BC08AE1F0
:1022800063E870E007C08BE16CE870E003C08CE1AC
:1022900065E970E00E94FD0E15C08DE16EE970E009
:1022A000F9CF812F67EA70E003C0812F60EB70E007
:1022B0000E94FD0E1E3031F01E3028F1812F895111
:1022C000853008F5812FB601A7010E94890B8AE7A6
:1022D00091E06A8149810E94260B6A816A5F8AE7E0
:1022E00091E049810E94260B49814A5F8AE791E08B
:1022F0006A810E94260B6A816A5F49814A5F8AE788
:1023000091E00E94260B1F5F1E3109F07ACF809169
:10231000CB018E3108F050C08091CB01BE016F5FC0
:102320007F4FAE014E5F5F4F0E94890B89818150C4
:1023300089838A8181508A8310E060919C01709129
:102340009D0180919E0190919F012AE030E040E044
:1023500050E00E94DA33653071058105910508F07F
:1023600011E08AE791E060E00E942C276981610F0B
:102370008AE791E04A810E94260B4A81410F8AE751
:1023800091E069810E94260B6981610F4A81485F53
:102390008AE791E00E94260B6981685F4A81410FBC
:1023A0008AE791E00E94260B1E5F1930F8F28AE757
:1023B00091E061E00E942C270F900F90CF91DF9168
:1023C0001F91FF90EF90DF90CF9008950F93809131
:1023D000D0018730F0F48091D0018F5F8093D001DD
:1023E0006091D00161708AE791E00E942C272091D2
:1023F0007E012D5F00917F010E5F8AE791E066E22A
:1024000040E00E94C5278AE791E061E00E942C2706
:102410001FC08091C401282F332727FD309537FF37
:1024200003C0309521953F4F205D8AE791E068E237
:1024300042E001E00E94632A20917E012D5F00911D
:102440007F010E5F8AE791E066E240E00E94FB2791
:102450000F91089581E591E00E94E51D8CE291E0E5
:1024600062E373E043E00E940024882319F0813086
:1024700041F404C081E08093B30109C01092B3011C
:1024800006C081E591E00E94EB1D80E00895109266
:10249000B4018091B301882379F08CE291E061ED81
:1024A00071E00E94DE1E0E94E50E0E94610E0E94F5
:1024B000020D0E94B20D23C08CE291E06BED71E041
:1024C0000E94DE1E0E94E50E0E94610E8091B40102
:1024D0008823C1F486E391E066E00E94C92C88233A
:1024E00089F461E070E080E090E00E945E2EEECF23
:1024F0008CE291E068E373E044E10E943E1E80912B
:10250000B40108958091B4018823C9F7F1CF0F93E6
:102510001F930CE211E0C80161ED71E00E94DE1E24
:10252000C80185960E94E51D81E01F910F910895D5
:102530000F931F930CE211E0C80161ED71E00E945E
:10254000DE1EC8016BED71E04AE00E942121C80146
:1025500085960E94E51D81E01F910F9108956F926D
:102560007F928F929F92AF92BF92CF92DF92EF9223
:10257000FF920F931F93CF93DF9362E070E080E0B0
:1025800090E00E9441326F5F6093CC018091CC015A
:102590000E946D078093CD0113E056EFA52E5FEFEB
:1025A000B52E43EFE42E4FEFF42E3BEFC32E3FEF5B
:1025B000D32E24E5822E9DE0792E80E3682EC5E19E
:1025C000D0E002E0902E8CE291E00E946820882307
:1025D000D1F386E391E064E00E94C92C882339F1AD
:1025E0008091B201813041F0813018F0823061F485
:1025F00008C00E94871202C00E9498128093B60100
:1026000005C00E942A12FACF1092B6018091B6013D
:10261000882351F087EB91E0612F0E94060A81E048
:1026200080930B011092CB018091B6013AC186E3F1
:1026300091E065E00E94C92C882341F486E391E093
:1026400066E00E94C92C882309F43AC181E591E033
:102650000E94EB1D80E025C181E591E00E94F11D03
:10266000133011F417E013C0115011C086E391E04C
:1026700062E045E00E94DD2C882349F081E591E08D
:102680000E94F11D173011F413E001C01F5F86E3B3
:1026900091E063E045E00E94DD2C882369F081E54C
:1026A00091E00E94F11D8091B20190E0019663E0FB
:1026B00070E00E94C73311C086E391E061E045E01D
:1026C0000E94DD2C882371F081E591E00E94F11DCC
:1026D0008091B201882321F081508093B20102C021
:1026E0009092B20180917E018A9D802D1124865D99
:1026F00080938301109284018AE791E06BE873E094
:102700000E94E3301092830180917F0180938401C5
:102710008AE791E060E873E00E94E33080917E01F7
:1027200090E09C012E9DC0012F9D900D3E9D900D2F
:1027300011248C5A9F4F62E070E00E94C73360936F
:1027400083018091840190917F01890F809384019E
:102750008AE791E06EE10E9406318091B201E82F94
:10276000F0E0EE0FFF1FE45BFC4F659174918AE788
:1027700091E00E94E3308AE791E06FE10E94063128
:102780001092830180917F0123E0829FC001112478
:10279000809384018AE791E06DE673E00E94E33064
:1027A00060917E016C9D602D11246C5A40917F01D7
:1027B00050E0440F551F440F551F8AE791E021E177
:1027C00001E00E94632A80917E01682D681B409180
:1027D0007F0150E0440F551F440F551F8AE791E0D9
:1027E00020E10E94632A80917E0190E0BC01660F87
:1027F000771F680F791F709561957F4F6C5A4091D4
:102800007F0150E0440F551F440F551F212F205DBD
:102810008AE791E00E94632A1092830180917F01F0
:1028200025E0829FC0011124809384018AE791E012
:1028300060E673E00E94E330E091CC0160917E019C
:10284000679DB0011124F0E0EE0FFF1FE35FFE4F24
:10285000208131818AE791E0409184010E94E22940
:102860001092830180917F01362D381B30938401B3
:102870008AE791E067E573E00E94E33080917E0192
:102880009E01281B3109C901880F991F880F991FC4
:10289000809383018AE791E062E573E00E94E33070
:1028A00092CEDF91CF911F910F91FF90EF90DF902B
:1028B000CF90BF90AF909F908F907F906F90089532
:1028C00086E391E060E045E00E94DD2C882309F07A
:1028D000C3CECCCE1092CF011092D00180910B01CB
:1028E000882339F087EB91E00E94540A10920B0183
:1028F00010C08091C601882361F087EB91E00E94AF
:10290000EA0987EB91E00E94540A87EB91E00E946C
:10291000410981E080930C010895DF93CF9300D0AB
:10292000CDB7DEB780910C01882379F11092CB01ED
:1029300005C08091CB018F5F8093CB016091CB016B
:1029400087EB91E00E9459079091C101891789F79F
:1029500087EB91E062EC71E00E94C409882351F496
:102960008CE291E06DED71E044E10E943E1E109218
:10297000CF010BC08091C40187FF07C08CE291E0BA
:102980006BEC71E048E20E943E1E8091CB01BE01DB
:102990006F5F7F4FAE014E5F5F4F0E94CD0B86E3AE
:1029A00091E062E043E00E94DD2C882359F081E54C
:1029B00091E00E94F11D8A818A3018F48F5F8A832A
:1029C00001C01A8286E391E060E043E00E94DD2CC2
:1029D000882359F081E591E00E94F11D8A818823C6
:1029E00011F0815001C089E08A838091E701853030
:1029F00008F4B3C086E391E063E04AE00E94DD2C76
:102A0000882309F4AAC081E591E00E94F11D80911C
:102A1000CB018F5F8093C20187EB91E062EC71E0A4
:102A20000E948D09882371F41092C20187EB91E016
:102A300062EC71E00E948D09882321F48091CB0122
:102A40008093C2018091C201BE016F5F7F4FAE01D2
:102A50004E5F5F4F0E94CD0B0FC08091E701853024
:102A600058F481E591E00E94F11D8981833018F4CA
:102A70008F5F898301C0198286E391E063E00E9441
:102A8000FB2C8093E70186E391E061E045E00E9442
:102A9000DD2C882359F081E591E00E94F11D8981A8
:102AA000882311F0815001C082E0898389816A8185
:102AB0000E94B80B8093CB0186E391E064E00E9412
:102AC000C92C8823A9F16091CB0187EB91E00E948A
:102AD00059079091C101891749F081E591E00E9461
:102AE000EB1D8CE291E069EB71E01FC08091CB019E
:102AF0008093C20187EB91E062EC71E00E943108A3
:102B0000882359F081E591E00E94E51D87EB91E073
:102B10000E943B091092CF010BC081E591E00E9419
:102B2000EB1D8CE291E06BEA71E044E10E943E1EF5
:102B300010920C018091B201823021F48091B30196
:102B40008823A1F08091C601882381F08091CF0174
:102B5000853060F00E946A1409C086E391E063E06A
:102B60000E94D32C882309F487CF77CF0F900F9042
:102B7000CF91DF910895FF920F931F9380910C01E5
:102B8000882309F447C09091C1018091CE01981724
:102B900009F440C09093CE0110E062E0F62E01E00F
:102BA0008CE291E00E9468208823D1F3112391F5F3
:102BB00086E391E064E00E94C92C882329F081E536
:102BC00091E00E94E51D11E08AE791E069E272E080
:102BD0000E94E33080917E0180938301F092820114
:102BE0009091CC018091C101891729F48AE791E085
:102BF00061ED71E004C08AE791E06BED71E00E9445
:102C0000E531009382018AE791E062E172E00E947F
:102C1000E330C6CF0E948D141F910F91FF9008954D
:102C200080910C01882361F087EB91E00E94DE0A1D
:102C3000882319F08091C20101C08EE18093CB01FD
:102C400010920C018091CF018A30F8F08091C6017A
:102C50008823D9F487EB91E00E94DE0A882329F0CB
:102C600087EB91E00E943B0907C08CE291E06EEE99
:102C700071E04FE00E943E1E8EE18093CB011092E6
:102C8000CF0108950E946A1408958091CF018E317A
:102C9000C8F708959091CD018091C101891719F469
:102CA0000E94101608950E948D1408958091B3011A
:102CB000882341F180910C01882321F00E94980D16
:102CC0000E948B0C0E949E0C882321F41092B40168
:102CD0001092B5019091CC018091C101891729F41E
:102CE0000E945E0D0E948D14089510920C010E94A6
:102CF000E20C0E94BD0C8823E9F00E94760D0E9430
:102D00006A1408950E94660E882361F48CE291E0B3
:102D100062E072E04AE00E943E1E1092B4011092FE
:102D2000B50108959091CD018091C101891711F4E9
:102D30000E948D1408950E946A1481E08093B50169
:102D400043C08CE291E00E9468208823E9F1609101
:102D5000CD0187EB91E00E948009882341F46091C6
:102D6000CC0187EB91E00E948009882399F11092B1
:102D7000B6010E941B0F08958091CF018F5F809351
:102D8000CF0186E391E066E00E94C92C882329F0F8
:102D900081E591E00E94EB1D08950E94EE0F0E94D4
:102DA000D7100E94E6118091B201813041F081304C
:102DB00018F0823049F406C00E944A1605C00E94ED
:102DC000BB1502C00E9456168091B501882309F0F8
:102DD000B8CF08958091CF018F3F71F6D2CF8CE2AA
:102DE00091E06BEF72E045E00E940024813099F0A1
:102DF00082301CF4882331F01BC0823099F083307C
:102E0000B9F413C08091B601882311F40E94AF1267
:102E10008091B60102C00E94AF12882389F00E94FF
:102E20009B1608950E94260C08950E94F10B0895A8
:102E30008CE291E065E073E049EB50E00E9462258E
:102E400008950E94EF1608950F931F930CE211E06E
:102E5000C8010E94C5268AE791E067ED79E00E94EB
:102E6000502AC80160EA73E049EB50E00E946225F5
:102E7000C8010E941D2080E58093DB018CE68093D1
:102E8000DC0181E68093DD0189E78093DE0185E640
:102E90008093DF0182E78093E00182E38093E10188
:102EA0001092E2011F910F910895882319F48CB5B7
:102EB000806202C08CB58F7D8CBD08959CB5937FD8
:102EC000982B9CBD08952CB5382F33702C7F322B56
:102ED0003CBD2DB590E0959587959595879581702A
:102EE0002E7F822B8DBD08958AE061E00E94312FF4
:102EF0008AE061E00E94F22E8CB580618CBD8CB5B9
:102F000080648CBD8DE061E00E94F22E8BE061E078
:102F10000E94F22E089581E080932D0260930A02B0
:102F200010922B0210922C0208952091090230E099
:102F300080910802281B3109C901089540910802B7
:102F400080910902481718F02FEF3FEF0AC0E42FD5
:102F5000F0E0E851FE4F8081282F30E04F5F409332
:102F60000802C9010895E091080280910902E8175A
:102F700018F0EFEFFFEF06C0F0E0E851FE4F808160
:102F8000E82FF0E0CF0108950895AC0120913002C0
:102F90003091310221153105E1F0909108028091C4
:102FA00009029817B0F090E008C0FA01EA0FFB1F81
:102FB0008081A851BE4F8C939F5FA92FB0E0A617C8
:102FC000B7079CF31092080260930902CB01F90144
:102FD00009950895E0912E02F0912F02309729F083
:102FE00010922B0210922C020995089570933102D1
:102FF00060933002089570932F0260932E0208951B
:10300000109235021092340288EE93E0A0E0B0E016
:103010008093360290933702A0933802B09339021E
:1030200087E191E090933302809332020895CF922A
:10303000DF92EF92FF920F931F93CF93DF937C0168
:103040006B018A0180912D028823A1F0C0E0D0E0BD
:103050000DC0D701ED91FC91D601AC0FBD1F0190C1
:10306000F081E02DC7016C9109952196C017D10719
:1030700080F304C0CB01642F0E946419C801DF9162
:10308000CF911F910F91FF90EF90DF90CF90089517
:10309000DF93CF930F92CDB7DEB7FC0169838091A8
:1030A0002D028823C9F080912C02803238F081E013
:1030B00090E09383828320E030E015C080912B0262
:1030C000E82FF0E0E55FFD4F998190838F5F80935B
:1030D0002B0280932C0205C0CE01019661E00E9474
:1030E000641921E030E0C9010F90CF91DF9108957C
:1030F0000F93062F80910A026BE072E040912C0240
:1031000021E00E940F1910922B0210922C021092B3
:103110002D020F91089561E00E94781808954132C0
:1031200008F040E2862F68EE71E00E94C618109207
:10313000080280930902089521E00E948F180895E3
:10314000109208021092090210922B0210922C0287
:103150000E941A1B08950F931F938C01862F0E94C3
:10316000C2188AEE97E10E94841985EC97E10E94CB
:103170007F19C8010E94A0181F910F9108950E9405
:10318000AB180895880F8093BA000895382F413204
:1031900010F040E042C080913E028823E1F791E0C8
:1031A00090933E02209340028FEF8093AB021092E7
:1031B00066024150409367024F5F90933F028091B7
:1031C0003F02330F832B80933F0280914102813075
:1031D00041F41092410280913F028093BB0085EC44
:1031E00001C085EE8093BC0080913E028130E1F306
:1031F00080916602841710F44091660220E030E06E
:103200000AC0FB01E20FF31FD901AA5BBD4F8C91ED
:1032100080832F5F3F4F2417A0F3842F08950F93CF
:103220001F93582F122F413210F081E04AC0809135
:103230003E028823E1F782E080933E020093400241
:103240008FEF8093AB021092660240936702A6E470
:10325000B2E0FB0102C081918D938E2F861B8417F3
:10326000D0F310923F0280913F02550F852B80933F
:103270003F0280914102813041F4109241028091DD
:103280003F028093BB0085EC01C085EE8093BC00BB
:10329000112321F080913E028230E1F38091AB0254
:1032A0008F3F11F480E00DC08091AB02803211F4A9
:1032B00082E007C08091AB02803311F084E001C04E
:1032C00083E01F910F910895482F613210F081E043
:1032D000089580913E02843011F082E00895609359
:1032E0008902A8E6B2E0842F9C01F90102C0819115
:1032F0008D938E2F841B8617D0F380E008959093D2
:1033000045028093440208959093430280934202C1
:1033100008951F920F920FB60F9211242F933F938F
:103320004F935F936F937F938F939F93AF93BF93CD
:10333000EF93FF938091B90090E0887F9070803682
:10334000910509F4F2C081369105CCF588329105DA
:1033500009F47BC089329105B4F48031910509F4F8
:103360006FC0813191053CF4009709F447C108977B
:1033700009F04FC165C08831910509F466C0809796
:1033800009F047C182C08034910509F4A4C081349A
:10339000910544F48033910509F482C0C89709F07F
:1033A00038C189C08035910509F489C088359105F7
:1033B00009F496C08834910509F02BC1AEC0883954
:1033C000910509F413C189399105ECF48837910509
:1033D00009F4ABC0893791054CF48836910509F49E
:1033E000A4C08037910509F014C19FC088389105A9
:1033F00009F4FCC08039910509F49DC0803891051D
:1034000009F007C198C0803B910509F4C6C0813B13
:1034100091054CF4803A910509F49FC0883A9105D2
:1034200009F0F7C0BAC0803C910509F4E3C0883CBC
:10343000910509F4DFC0883B910509F0EAC0C2C0DC
:1034400080913F028093BB00CFC090916602809133
:103450006702981768F490916602E92FF0E0EA5B42
:10346000FD4F80818093BB009F5F90936602BCC03C
:1034700080914002882309F44BC085ED8093BC0005
:103480008091BC0084FDFCCFC2C080E28093AB027F
:1034900085ED8093BC008091BC0084FDFCCFB7C05B
:1034A00080E38093AB0285ED8093BC008091BC00EB
:1034B00084FDFCCFACC088E38093AB029BC08091BD
:1034C00066029091BB00E82FF0E0EA5BFD4F90832D
:1034D0008F5F80936602909166028091670282C03E
:1034E000809166029091BB00E82FF0E0EA5BFD4F0F
:1034F00090838F5F8093660280914002882341F021
:1035000085ED8093BC008091BC0084FDFCCF7FC022
:1035100081E08093410284EA6EC085ED8093BC0017
:103520008091BC0084FDFCCF72C083E080933E029A
:103530001092AA0259C08091AA02803208F056C0A7
:103540008091AA029091BB00E82FF0E0E657FD4F72
:1035500090838F5F8093AA0247C08091AA02803235
:1035600030F4E091AA02F0E0E657FD4F108285EDBD
:103570008093BC008091BC0084FDFCCF10923E0281
:103580006091AA02E0914402F09145028AE892E03B
:1035900070E009951092AA022DC084E080933E024B
:1035A0001092880210928902E0914202F091430247
:1035B000099580918902882329F481E0809389020A
:1035C0001092680290918802E92FF0E0E859FD4FCF
:1035D00080818093BB009F5F9093880290918802C6
:1035E00080918902981710F485EC01C085E88093DA
:1035F000BC000FC085EC8093BC0009C01092AB02E8
:1036000085ED8093BC008091BC0084FDFCCF1092BE
:103610003E02FF91EF91BF91AF919F918F917F916A
:103620006F915F914F913F912F910F900FBE0F902F
:103630001F90189510923E0281E0809340021092F4
:10364000410282E161E00E94312F83E161E00E944A
:10365000312FE9EBF0E080818E7F808380818D7F48
:10366000808388E48093B80085E48093BC0008954B
:10367000FC01662371F4178A158A14A213A2108E16
:103680001092B0021092AF021092AD021092B400EC
:10369000118208950F931F93CF93DF93EC018B0159
:1036A000442371F460E00E94381B1E870D871B8A3B
:1036B0001A8A81E0898389E08E8B198E1B8E1D8E7C
:1036C000DF91CF911F910F910895CF93DF93EC017C
:1036D000662339F58881882321F18981882309F5BA
:1036E000898590E0880F991FEF81F885E80FF91F11
:1036F000859194912FEF8F3F920711F4188211C09A
:103700009C8790E0880F991FEA85FB85E80FF91FD9
:1037100065917491CE0140E00E944A1B89858F5FBC
:103720008987DF91CF91089560E00E94651B08951D
:1037300060E00E94381B08950F93DC01002309F01C
:1037400069C0623009F443C0633030F4662359F035
:10375000613009F05FC00DC0633009F444C06430CB
:1037600009F058C04CC04B3008F04AE056964C93D4
:1037700051C0842F90E0880F991F1F962D913C9186
:103780005097280F391FF9018591949190969C9339
:103790008E935F97FC014591549114968C911497E8
:1037A000849F602D112491966C939197252F332738
:1037B000862F90E02817390708F4652F14968C910E
:1037C0001497689F802D112492968C9323C0149691
:1037D0008C911497489F802D112459968C9359975A
:1037E0005A962C9317C014968C911497489F802D4D
:1037F00011245B968C935B975C962C930BC014966C
:103800008C911497489F802D11245D968C935D9721
:103810005E962C930F9108950F93CF93DF93EC0155
:10382000662309F07BC08981882309F477C08D89DC
:10383000882309F073C0EA89FB89EE0FFF1F4D85CD
:103840005E85E40FF51F259134912115310509F0AE
:1038500049C08989813031F41B8A1A8AFA0125917D
:10386000349140C019828881882379F0CE0160E0CC
:103870000E94651B8A899B89880F991FED85FE85AB
:10388000E80FF91F259134912DC01F8A1D8A1CA2B3
:103890001BA2188E1092B0021092AF021092AD02CD
:1038A0001092B4003BC006E0369527950A95E1F7E3
:1038B0006F70422F4F71B5E036952795BA95E1F7B5
:1038C0002051CE0100E00E949C1B8A899B890196B1
:1038D0009B8B8A8B880F991FED85FE85E80FF91F5A
:1038E00025913491B901769567957695679520FD78
:1038F000DACF862F8F738C8B8C81839F802D112440
:103900008D8B1DA21CA21BA281E08F8B8093AD0228
:10391000188E8A899B8901969B8B8A8BDF91CF9128
:103920000F91089560E00E940C1C0895CF93DF93DF
:10393000EC01662309F0E9C08F89882309F4E5C00A
:103940008D89882371F41F8A1D8A1CA21BA2188EE0
:103950001092B0021092AF021092AD021092B40019
:10396000D4C081508D8B8DA1882309F044C08BA1D8
:103970009CA10196880F991FEF8DF8A1E80FF91F00
:1039800085919491282F27702EA3AC0173E0569552
:1039900047957A95E1F79A0136952795892F9927CA
:1039A000869586958FA32F738C81289F202D1124B7
:1039B0002DA341704093B1028BA19CA101969CA3C1
:1039C0008BA329A130E082179307A8F08AA188234E
:1039D00029F0281B31093CA32BA30DC01F8A1D8A87
:1039E0001CA21BA2188E1092B0021092AF0210926D
:1039F000AD021092B4008DA181508DA3988D9F5F70
:103A0000988F2FA18C89280F8C85280F2A836B8D86
:103A1000662369F0892F992787FD909570E00E94B1
:103A2000C7338C8D869F802D1124820F8A838A81D3
:103A300090E0CB966BE370E00E94C7338A832E89B7
:103A40002B83698D662379F0888D772767FD7095C4
:103A5000992787FD90950E94C7338A8D869F802D78
:103A60001124820F8B836D8D662399F0888D9927A1
:103A700087FD909570E00E94C733CB0162E070E053
:103A80000E94C7339E8D899F802D11249B81890FB1
:103A90008B838B818A300CF089E087FD80E08B83FB
:103AA0008C898F3309F41B82F894EA81F0E0E159A4
:103AB000F44FE491E093AE022D8130E08B819927A1
:103AC00087FD9095A901489F9001499F300D589F0F
:103AD000300D112488A590E0A901489F9001499FCD
:103AE000300D589F300D11248EA1992787FD909598
:103AF000AC01249FC001259F900D349F900D11248F
:103B00008093AF028093B0027894DF91CF910895B3
:103B100060E00E94961C08956091AF02662381F1D7
:103B20008091AC028F5F8093AC029091AE028917B6
:103B300038F130E08091AD02882309F431E0309310
:103B4000AD021092AC028091B1028823A9F080915D
:103B50000D0123E4829FC0011124895B80930D0134
:103B600090E070E00E94B3338093B00205C0809172
:103B7000B0028093B40008953323C9F780E0F9CFF1
:103B800008951F920F920FB60F9211242F933F9317
:103B90004F935F936F937F938F939F93AF93BF9355
:103BA000EF93FF930E948C1DFF91EF91BF91AF9116
:103BB0009F918F917F916F915F914F913F912F9145
:103BC0000F900FBE0F901F90189567E67BE040E0C6
:103BD0000E944A1B08956FE57BE040E00E944A1B6B
:103BE000089569E57BE040E00E944A1B0895FC01CE
:103BF000862F668170E06F5F7F4F992787FD9095D4
:103C00000E94C733858308950F93FC0181E084836C
:103C100084E080A78AEA9BE0908B8787CF0161E0F0
:103C200040E020E000E00E949C1B83E061E070E047
:103C30000E94FA2FE1EBF0E08081887F8160808331
:103C4000F89410928000E1E8F0E010821092850074
:103C50001092840088E191E090938900809388001D
:103C6000808188608083808181608083EFE6F0E0DE
:103C700080818260808378940F910895FC01ED57D4
:103C8000FF4F61937193445F40830895CF93DF9317
:103C9000DC01E0E8F7E785919491ED01C75ADF4F29
:103CA000AD0141595F4F8150904C09F04EC0E6E99B
:103CB000F7E7E491E883E7E9F7E7E4911496EC93FA
:103CC0001497E8E9F7E7E4911596EC931597E9E97D
:103CD000F7E78591949117969C938E931697EBE94D
:103CE000F7E78591949119969C938E931897EDE937
:103CF000F7E7E4919B96EC939B97EEE9F7E7E49165
:103D00009A96EC939A97EFE9F7E7E491EA01E88352
:103D1000E0EAF7E7859194915D969C938E935C978A
:103D2000E2EAF7E7859194915F969C938E935E9774
:103D3000E4EAF7E78591949191969C938E939097FE
:103D4000E6EAF7E78591949132C08CE38883149674
:103D50001C9214972FEF15962C93159780E293E001
:103D600017969C938E93169784ED93E019969C93E7
:103D70008E93189781E09B968C939B979A968C9341
:103D80009A97FA0120838CEA9DE05D969C938E932E
:103D90005C978EED9DE05F969C938E935E9784E793
:103DA0009EE091969C938E9390978CE39FE09396E0
:103DB0009C938E939297DF91CF910895E0E8F7E777
:103DC000859194918150904C51F4DB01EBE8F7E739
:103DD00084918D93319687E7E539F807C9F70895FF
:103DE000EF92FF920F931F93CF93DF937C018C018F
:103DF000025B1F4FC8010E94D82BC8016BED7BE00E
:103E00000E94E330C8010E94982B83E00E94631750
:103E100080E091E0EEEFFFE3099584E590E0E80EA5
:103E2000F91EF7011082C80166EB7BE00E942E317B
:103E3000C8010E94982BE701CA54D040CE010E94CD
:103E4000032DCE0164E00E94C92C882339F462E37B
:103E500070E080E090E00E945E2EF0CFDF91CF9185
:103E60001F910F91FF90EF9008950F931F93CF93A1
:103E7000DF93EC018C01025B1F4FC80161E040E061
